:100000002828A301A200FF30A207031CA307031C9A
:1000100023280330A100DF300F200328A101E83E90
:10002000A000A109FC30031C1828A00703181528FC
:10003000A0070000A10F152820181E28A01C2228A8
:100040000000222808008313831203130000080015
:1000500007309F00831685011F30860083128612A9
:10006000061386138501A501A401861838284228A5
:1000700006193B28522886193E286628061A412868
:10008000A6282E280613861386168501A501A4012D
:1000900006184B282E2806194E2852288619512852
:1000A00066284228861286130617051185158510C5
:1000B00005108513A501A40106185F282E288618AF
:1000C0006228422886196528662852288612061357
:1000D000861705158511A501A40185140510851342
:1000E000FA300120061875282E288618782842280C
:1000F00006197B285228851005148513FA30012033
:10010000061883282E28861886284228061989284A
:100110005228851005108517FA30012006189128FD
:100120002E288618942842280619972852288510C8
:1001300005148513FA30012006189F282E288618EA
:10014000A22842280619A52852286D28A501A40135
:1001500002302502031CB228031DC4286330240288
:100160000318C428061EB5282E288618B828422849
:100170000619BB2852288619BE286628643001203B
:10018000A40A0319A50FA8288612061386130515BD
:100190008511851405108513FA300120061ED1281B
:1001A0002E288618D42842280619D72852288619BE
:1001B000DA286628851005148513FA300120061EFA
:1001C000E2282E288618E52842280619E828522811
:1001D0008619EB286628851005108517FA3001204E
:1001E000061EF3282E288618F62842280619F92814
:1001F00052288619FC286628851005148513FA30C4
:100200000120061E04292E288618072942280619CF
:0C0210000A29522886190D296628C928E1
:02400E00183F59
:00000001FF
